:1000000000308A003F2900000A108A100A11820776
:1000100028340C34013406340A108A100A1182077D
:10002000413454342B3443344D3447344C343D3410
:1000300031340D3400342D3084008313000803194B
:1000400032280130F800BF30F7006400F70B252894
:10005000F80B23284A30F700F70B2C280000640027
:10006000800B212800340708F039B40033080F3919
:100070003404870006148316061064002030F7004D
:10008000F70B4028432883120610831606108312AC
:100090000034B108031D4E2886104F28861483169D
:1000A00086108312B20E3208B3003320B20E32082B
:1000B000B300332064004230F700F70B5D280034B2
:1000C0001430AD001B20F030831687058312861094
:1000D0008316861083120610831606108312AA0157
:1000E0002A08023C031C7C280230AD001B20033090
:1000F000B3003320AA0A702864000C30F700F70B15
:100100007F2882280230B300332064000C30F700CF
:10011000F70B88288B28AA012A08023C031C9C287C
:100120002A080420AB00B1012B08B200492002309C
:10013000AD001B20AA0A8C28902901302E02FC3E1B
:100140000318AF28043EBA28AF01AF284030AF00F3
:10015000AF281430AF00AF285430AF00AF280130C3
:100160002D02AF072F088038B000B1013008B2006F
:10017000492000340A108A100A118207A428A628F0
:10018000A928AC282C080C3A0319D028063A0319E0
:10019000D828073A0319DE28053A0319E328E82886
:1001A000B1010130B20049200230AD001B20F4281B
:1001B0000130AD000230AE009D20F4280130AD00CA
:1001C000AE009D20F428B1011030B2004920F4287F
:1001D0002C081F3C031CEE280730AC050130B10091
:1001E0002C08B2004920F42800342D08F8012C0214
:1001F0000318FD282C08F7000929F7010830AE0084
:10020000AC0DF70D2D0877020318F700F80DAE0BB3
:100210000029003478082A08AC006430AD00F520CD
:100220007708AA0078083030031D1D29AB1C24294B
:10023000AB1924292B1A20302029AB112B122B1497
:10024000F8077808AC00C2202A08AC000A30AD00DC
:10025000F5207708AA0078083030031D3529AB193E
:1002600039292B1C39292B1A2030F8077808AC00C3
:10027000C2203030AA072A08AC00C2200034840112
:1002800083131F3083050C3083169900A630980025
:1002900090308312980083161F149F141F159F110E
:1002A00007309C00FF308312A00083161F149F1498
:1002B0001F159F1183121F108316091283129412A7
:1002C000A0122008831687008312201620088316A8
:1002D00087008312A0112008831687000130831243
:1002E00094000030831694000108C7390838810053
:1002F000831290010030F8009200003083169200C3
:1003000007309C00050864000230F700F70B8629CF
:1003100089291C0883120D1383169D0183126028FE
:10032000AA012A080C20AA0AF70077080C1E9629B1
:1003300099000A302A02031D912921308400831379
:100340008403840A8C1EA2291A0880000D30000242
:10035000031DA12980018C1EAB291A088C1EAE2911
:100360001A082130840083138403840A8C1EB62962
:100370001A0880000D300002031DB5298001A90173
:100380002908363C031CC9298C1EC4291A08A90A4D
:10039000C0292130840083138403840A8C1ECE2953
:1003A0001A0880000D300002031DCD298001213084
:1003B00084008313003000040319EE29AB01040804
:1003C000AA002B10831B2B140008AC00C2202A08A3
:1003D000840083132B188317840ADA290A30AC00AF
:1003E000C220A108031DF6293030A2003030A1023E
:1003F000A2022108093C0318FF290730A1022208A4
:10040000093C0318052A0730A202A10EF030A1050D
:100410002208A104A308031D0F2A3030A4003030A5
:10042000A302A4022308093C0318182A0730A302D8
:100430002408093C03181E2A0730A402A30EF0303A
:10044000A3052408A304A508031D282A3030A6000C
:100450003030A502A6022508093C0318312A0730CE
:10046000A5022608093C0318372A0730A602A50E64
:10047000F030A5052608A504A708031D412A303041
:10048000A8003030A702A8022708093C03184A2A0E
:100490000730A7022808093C0318502A0730A80291
:1004A000A70EF030A7052808A7042108AA001B30D2
:1004B000AB000A212030AC00C2202308AA001B3068
:1004C000AB000A212030AC00C2202508AA001B3056
:1004D000AB000A212030AC00C2202708AA001B3044
:0604E000AB000A216300DD
:02400E00393F38
:00000001FF
